:1000000019C033C032C031C030C02FC02EC02DC087
:100010002CC02BC064C029C028C028C026C025C061
:1000200024C023C022C021C020C01FC01EC01DC0CC
:100030001CC01BC011241FBECFEFD4E0DEBFCDBF5C
:1000400011E0A0E0B1E0E8E0FBE002C005900D9215
:10005000A033B107D9F711E0A0E3B1E001C01D92D0
:10006000AE35B107E1F7F0D14DC5CACF1F920F925F
:100070000FB60F9211248F939F9380915601909108
:10008000570101969093570180935601789480917F
:100090003A0190913B01019690933B0180933A0184
:1000A00080914D01882339F080914D0181508093DA
:1000B0004D015D9A01C05D98809134018F5F8093FE
:1000C00034018E3128F01092340181E0809339019F
:1000D0009F918F910F900FBE0F901F9018951F92B8
:1000E0000F920FB60F9211242F933F938F939F93EC
:1000F000AF93BF938091300190913101A091320173
:10010000B09133010196A11DB11D809330019093F0
:100110003101A0933201B093330120915D01213070
:1001200069F58093480190934901A0934A01B093E7
:100130004B0120918600309187003093530120932A
:10014000520120915601309157013093550120936F
:100150005401B09B10C0209152013091530137FDE2
:100160000AC020915401309155012F5F3F4F3093C9
:1001700055012093540122E020935D01B59B0DC0F1
:100180000196A11DB11D8093300190933101A09380
:100190003201B093330180E286BBBF91AF919F9152
:1001A0008F913F912F910F900FBE0F901F90189538
:1001B00082E306C0E1EEF4E03197F1F700C0000001
:1001C0008150C0F70895419A84E08A95F1F70000C4
:1001D0004198089595B1869586958C73937C892B6B
:1001E00085B9F1DF0895F6DF83ED90E30197F1F72C
:1001F00000C0000008951F93182F662311F0409A45
:1002000001C04098812FE6DF812F8295807FE2DF59
:1002100081EE94E00197F1F700C000001F9108956E
:1002200061E0E9DF0895CF93DF93EC0101C0F8DFCF
:1002300089918823E1F7DF91CF910895AF92BF9222
:10024000CF92DF92EF92FF920F931F936B017C018D
:10025000142F7D2D9F2D2FE632E143E85AE3EBD397
:1002600087FF07C013E000E0FF24EE24DD24CC2448
:1002700087C0112311F413E019C060E070E080E83A
:100280009FE32C2D3D2D4E2D5F2D8AD26B017C01DD
:1002900015E00CC06C2D7D2D8E2D9F2D20E030E0C3
:1002A0004AE754E4CCD36B017C011F5F6C2D7D2D9C
:1002B0008E2D9F2D20E030E040E85FE36DD287FD7A
:1002C000E9CF0CC06C2D7D2D8E2D9F2D2FE632E1B8
:1002D00043E85AE3B4D36B017C0111506C2D7D2DA2
:1002E0008E2D9F2D20E030E04AE754E4A4D387FF11
:1002F000E9CF00E00CC06C2D7D2D8E2D9F2D2DECB7
:100300003CEC4CEC5DE39BD36B017C010F5F6C2DEF
:100310007D2D8E2D9F2D20E030E040E251E48BD3E7
:1003200087FFE9CF6C2D7D2D8E2D9F2D2CEA35EC8E
:1003300047EA56E3CDD1F62EE72ED82EC92EA701D7
:100340009601652F742F832F922F20E030E040E23A
:1003500051E471D38823A4F0A7019601652F742F6F
:10036000832F922F2DEC3CEC4CEC5DE368D3F62E02
:10037000E72ED82EC92E0F5F033014F0115000E085
:10038000BB24A7019601652F7E2D832F9C2D70D253
:10039000A62E862F805D44DFB01611F48EE240DF7A
:1003A000B39486E0B816D1F06A2D772767FD709573
:1003B000872F972F90D29B01AC01D701F6016B2FAD
:1003C0007E2D8F2F9C2D83D120E030E040E251E440
:1003D00036D3F62EE72ED82EC92ED3CF80E220DFDB
:1003E000812F992787FD9095880F991F880F991F56
:1003F000885F9E4F18DF80E213DF1F910F91FF90FF
:10040000EF90DF90CF90BF90AF90089560E0F3DE63
:100410000895CEDE80E3E7DE80E3E5DE80E3E3DE21
:1004200080E2E1DE88E2F2DF8CE0F0DF81E0EEDF07
:10043000BFDE80E8EBDF80E091E0F5DE80ECE6DF18
:1004400084E091E0F0DE08958F929F92AF92BF9288
:10045000CF92DF92EF92FF920F931F9311E015B9A5
:100460008CE384B983E087B980E28AB98CE18BB9E7
:1004700087E085BDCEDF10924C0180B7846080BFDD
:1004800010925D01109258011093810081E28093D7
:100490006F0078940EE180913901882319F1109250
:1004A000390186B5A89B02C015BB8FEF16BC909191
:1004B0005801992361F08930A8F480B7846080BF27
:1004C00010935D0110924C01109258010BC08131C4
:1004D00048F01093580180B7887F80BF10935D016A
:1004E00010924C0180916F008E7F80936F008091FD
:1004F0005D01882369F480913A0190913B01843633
:10050000910530F010935D0110923B0110923A0179
:1005100080916F00816080936F0080915D018230D7
:1005200009F0B9CF80915401909155012091520169
:1005300030915301A0E0B0E0DC019927882740E02A
:1005400050E0820F931FA41FB51F80934E0190931C
:100550004F01A0935001B093510180914E019091B1
:100560004F01A0915001B091510120913C01309177
:100570003D0140913E0150913F01821B930BA40B22
:10058000B50B8093590190935A01A0935B01B093EE
:100590005C0180914E0190914F01A0915001B0916A
:1005A000510180933C0190933D01A0933E01B09393
:1005B0003F018091480190914901A0914A01B09179
:1005C0004B012091400130914101409142015091F5
:1005D0004301821B930BA40BB50B809344019093B2
:1005E0004501A0934601B093470180914801909145
:1005F0004901A0914A01B0914B0180934001909331
:100600004101A0934201B093430110925D0180919A
:100610004C01882309F458C000934D0160914401B6
:10062000709145018091460190914701C090590118
:10063000D0905A01E0905B01F0905C014AD120E833
:1006400036E948E95BE4FBD14B015C01C701B60127
:1006500040D19B01AC01C501B401A2D0262F372F98
:10066000482F592F2093350130933601409337019D
:100670005093380120915801222369F020E030E0A6
:1006800040E854E4DCD160933501709336018093E7
:1006900037019093380184E8B9DE6091350170919B
:1006A0003601809137019091380140E0C7DD84EC3C
:1006B000ADDE6091350170913601809137019091E6
:1006C000380141E0BBDDE7CE10934C01E4CE505839
:1006D000BB27AA270ED075C166D130F06BD120F0B0
:1006E00031F49F3F11F41EF45BC10EF4E095E7FB7B
:1006F00051C1E92F77D180F3BA17620773078407D6
:10070000950718F071F49EF58FC10EF4E0950B2E4D
:10071000BA2FA02D0B01B90190010C01CA01A00153
:100720001124FF27591B99F0593F50F4503E68F1AE
:100730001A16F040A22F232F342F4427585FF3CFEF
:10074000469537952795A795F0405395C9F77EF4C0
:100750001F16BA0B620B730B840BBAF09150A1F009
:10076000FF0FBB1F661F771F881FC2F70EC0BA0F8F
:10077000621F731F841F48F4879577956795B79517
:10078000F7959E3F08F0B3CF9395880F08F099270F
:10079000EE0F979587950895D9D008F481E00895D4
:1007A0000CD00FC107D140F0FED030F021F45F3FF4
:1007B00019F0F0C0511139C1F3C014D198F3992345
:1007C000C9F35523B1F3951B550BBB27AA27621715
:1007D0007307840738F09F5F5F4F220F331F441F5A
:1007E000AA1FA9F333D00E2E3AF0E0E830D0915092
:1007F0005040E695001CCAF729D0FE2F27D0660F7F
:10080000771F881FBB1F261737074807AB07B0E8BD
:1008100009F0BB0B802DBF01FF2793585F4F2AF0D3
:100820009E3F510568F0B6C000C15F3FECF3983EB3
:10083000DCF3869577956795B795F7959F5FC9F730
:10084000880F911D9695879597F90895E1E0660FB9
:10085000771F881FBB1F621773078407BA0720F032
:10086000621B730B840BBA0BEE1F88F7E09508959B
:1008700004D06894B111D9C00895BCD088F09F57B6
:1008800090F0B92F9927B751A0F0D1F0660F771FDC
:10089000881F991F1AF0BA95C9F712C0B13081F0BC
:1008A000C3D0B1E00895C0C0672F782F8827B85F04
:1008B00039F0B93FCCF3869577956795B395D9F71D
:1008C0003EF490958095709561957F4F8F4F9F4F27
:1008D0000895E89409C097FB3EF490958095709533
:1008E00061957F4F8F4F9F4F9923A9F0F92F96E97C
:1008F000BB279395F695879577956795B795F111F1
:10090000F8CFFAF4BB0F11F460FF1BC06F5F7F4F8D
:100910008F4F9F4F16C0882311F096E911C077239F
:1009200021F09EE8872F762F05C0662371F096E8A8
:10093000862F70E060E02AF09A95660F771F881F77
:10094000DAF7880F9695879597F90895990F00081B
:10095000550FAA0BE0E8FEEF16161706E807F90791
:10096000C0F012161306E407F50798F0621B730B2C
:10097000840B950B39F40A2661F0232B242B252BAD
:1009800021F408950A2609F4A140A6958FEF811D50
:10099000811D089597F99F6780E870E060E00895F1
:1009A0009FEF80EC089500240A9416161706180687
:1009B0000906089500240A94121613061406050663
:1009C0000895092E0394000C11F4882352F0BB0FF4
:1009D00040F4BF2B11F460FF04C06F5F7F4F8F4F57
:1009E0009F4F089557FD9058440F551F59F05F3F92
:1009F00071F04795880F97FB991F61F09F3F79F041
:100A000087950895121613061406551FF2CF4695C2
:100A1000F1DF08C0161617061806991FF1CF869544
:100A20007105610508940895E894BB276627772728
:100A3000CB0197F908958ADF08F48FEF08950BD062
:100A4000C0CFB1DF28F0B6DF18F0952309F0A2CFB0
:100A5000A7CF1124EACFC6DFA0F3959FD1F3950F5E
:100A600050E0551F629FF001729FBB27F00DB11D32
:100A7000639FAA27F00DB11DAA1F649F6627B00DC2
:100A8000A11D661F829F2227B00DA11D621F739FAB
:100A9000B00DA11D621F839FA00D611D221F749FB9
:100AA0003327A00D611D231F849F600D211D822F00
:100AB000762F6A2F11249F5750408AF0E1F0882347
:100AC0004AF0EE0FFF1FBB1F661F771F881F915054
:100AD0005040A9F79E3F510570F05CCFA6CF5F3F15
:100AE000ECF3983EDCF3869577956795B795F79587
:100AF000E7959F5FC1F7FE2B880F911D969587950F
:080B000097F90895F894FFCF66
:100B0800462E3A00502E3A0047487A004D487A005F
:100B18006B487A00487A20006D487A0073656B004C
:100B28006D732000757320006E73200070732000B1
:00000001FF
